:100000002E288001840AFF3E031D01282928A30110
:10001000A200FF30A207031CA307031C29280330FA
:10002000A100DF3015200928A101E83EA000A109A8
:10003000FC30031C1E28A00703181B28A007000083
:10004000A10F1B2820182428A01C282800002828DD
:10005000080083138312031300000800073099007F
:100060008501FE3083168500383096008B138B1582
:10007000203084004030831201205928851A24142E
:10008000851E2410051AA414051EA4100508A60038
:100090000B106300851A2514851E2510051AA5145A
:1000A000051EA510240825020319722805148316BD
:1000B000051083128519712805108316051001306B
:1000C0008312A300F4300820051483160510C830ED
:1000D00083120720051083160510143083120720A1
:1000E00072285A280230A300583008208519BC28ED
:1000F00005108316051001308312A300F430082088
:10010000051483160510C8308312072005108316C6
:100110000510C83083120720051483160510C83057
:100120008312072005108316051014308312072050
:1001300085199B28982814300720851DBB280508A1
:10014000A6000B1063008519BA2805108316051048
:1001500001308312A300F430082005148316051023
:10016000C83083120720051083160510143083123F
:100170000720BB289D28BD283E283E286300BE28B6
:02400E00843FED
:00000001FF
